:020000020000FC
:0200000084C0BA
:020004002AC010
:100008004BC0000101010202030405070A0D121882
:10001800222D000001010101010102020202020376
:10002800030404050607080A0B0D0F1215181D22F4
:10003800282D070707070404040401070305000621
:100048000204FF0FFF0FFF0F1FFF1F1F1FFFFF0FF0
:10005800FFFF4B990AC01AB957B84A99FECF77B82B
:100068007AB8F1E042E04CBB1895E6B1EF734F99CE
:100078000AC0F09904C0F1E050A010A9F2CFF3E053
:1000880050A010A9EECFEF3319F0EE3319F0E9CFF5
:10009800F098E7CFF09AE5CF46B14F734A991BC065
:1000A80059B07FB658204529542E5094F1E010815C
:1000B800F099F3E050A24123152D182110AB408B85
:1000C800ED3021F4F09B3068F09900687FBE77240A
:1000D800F1E0FCBB1895E42F4E990AC0F09904C0D2
:1000E800F1E050A010A9F4CFF3E050A010A9F0CF90
:1000F800EF3319F0EE3319F0EBCFF098E9CFF09A1F
:10010800E7CFF89400E00093600008ED0093340016
:1001180000E80093610008ED0093340000E00093CC
:10012800610008ED0093340004E00093050100EE3F
:10013800009366000FEF0A95F1F703E000930701BB
:100148000FE70093080100E80093200000C005B7FE
:10015800046005BF0FEF0DBF08E00EBF00E8009375
:10016800500000E80FBDF098F198772400EC802E3D
:1001780001E2D02E0FEF502E182DFF24DFEF20E1E3
:10018800E0E1F1E080A2008B71922A95D9F7B2E004
:10019800A0E1EAE3F0E020E1AED1A0E2EAE0F0E09D
:1001A80020E1A9D1A0E3EAE1F0E020E2A4D1AA2766
:1001B800B1E0EAE4F0E020E19ED120E1E0E1F3E003
:1001C80080A2008B71922A95D9F720E1E0E6F2E04F
:1001D80071922A95E9F7F1E0EE276F2E7092890067
:1001E8007092880070928B0070928A00219A229AED
:1001F80000240027009380000027009385000093C7
:10020800840007E000938100002704BD002706BD95
:1002180001E005BB01E005BDA0EDB7E005B300FFB7
:10022800FDCF01E005BB1197C9F700270093250012
:10023800009381004091840050918500002700932D
:10024800850000938400442311F45523F1F060E005
:1002580070E82EE3A42FB52FB695A7956A0F7B1FDC
:10026800271D88279927222319F46417750738F062
:10027800641B750B27098395B1F79395F4CF8150CB
:100288009040992311F4C82F009402EA009380004B
:1002980009E1009381002DEA002009F02C2F7092CB
:1002A8008700209386000FE00093690003E00CBBF1
:1002B80003E00DBBE0E13327002700244424112488
:1002C8002224AA24282D782D992466273324AA27A6
:1002D800BB2788279927CC24BB24D4E0CCE602E0AE
:1002E800088300E00983D4E21880D2E07894C6B38A
:1002F800C0FFFDCFC6BB3A94AAF4309016015091C6
:10030800160335160CF4352E3A9466946E2CF79431
:10031800E79438630863E0FE377CE0FE077C660CF0
:100328006E24669437FF06C0C0911D0198882FE19E
:100338003F770CC097FC13C001970CF081F42A9505
:100348002AF42FE191FC9F2692FC982880911B01AA
:1003580090911C01C22F5FE190FEC527C8A807FF36
:1003680006C0C0911D0368897FE10F770CC067FD47
:1003780013C011970CF081F47A952AF47FE161FD9E
:100388006F2762FD6829A0911B03B0911C03C72F3A
:100398005FE160FFC527B8A8F19B2CC0D1E2C0E699
:1003A8000880D0922100019B05C0C0E10880D0924E
:1003B80021003F27C0E62882C2E60880D0922100AB
:1003C800019B06C0C2E10880D092210052E0352787
:1003D800C2E62882C4E60880D0922100019B06C0AC
:1003E800C4E10880D092210054E03527C4E6288271
:1003F800F19831C0D1E2C6E60880D0922100019B75
:1004080007C0D3E2C0E10880D09221000F27D1E2D3
:10041800C6E62882C8E60880D0922100019B08C061
:10042800D3E2C2E10880D092210052E00527D1E250
:10043800C8E62882CAE60880D0922100019B08C03D
:10044800D3E2C4E10880D092210054E00527D1E22C
:10045800CAE62882F19A50911701532BC52FCC0F69
:10046800C2955C23D2E0C09118010C2CC4FF08A0EF
:1004780050FF0024C09119014C2CC4FF48A051FF23
:100488004424C0911A011C2CC4FF18A052FF112447
:10049800C42D46944694C4194694C4190C0E1C0ED7
:1004A80050911703502BC52FCC0FC2955C23C091D8
:1004B80018032B2CC4FF28A050FF2224C091190335
:1004C8004B2CC4FF48A051FF4424C0911A03AB2C05
:1004D800C4FFA8A052FFAA24C42D46944694C41968
:1004E8004694C4192C0EAC0E020C1A0C009288000B
:1004F80010928A00FCCE05910D932A95E1F7089594
:00000001FF
